:1000000012C02AC418951895189518951895189522
:100010001895189518951895189518951895189578
:100020001895189518958FE58DBFC8E3E6EF4E2E0D
:1000300084E08EBFD4E0F3E05F2E66248FEF84BBB4
:100040008FEF87BB80E088BB8A988B98E894A2E307
:10005000B0E08C9182F98C93E894A2E3B0E08C91AB
:1000600083F98C93A2D385B7836085BF8BB78064F7
:100070008BBF7894B99ABA9A81EA8FBD81E08EBD20
:10008000BB9A81E685BDB99ABA9ABB9A80E090E0A6
:1000900090934B0080934A0080E090E09093490059
:1000A0008093480080E083BD84E690E090934B000D
:1000B00080934A0084E690E0909349008093480042
:1000C00084EF91E0B4D388EC90E090934B00809360
:1000D0004A0088EC90E0909349008093480084EFB8
:1000E00091E0A5D380E090E090934B0080934A008C
:1000F00080E090E0909349008093480084EF91E085
:1001000096D380E090E0A2EAB0E08D939C93A0E3C8
:10011000B0E00C9103FB00270EF401E040E004176F
:1001200009F00EC0A2EAB0E072D3A2EAB0E00D91ED
:100130001C91083E53E0150709F001C036D3E7CF04
:10014000AFE9B0E00C9107FB00270EF401E041E0BD
:10015000041709F0EEC0AFE9B0E00C9104FB0027F2
:100160000EF401E041E0041709F007C0A9E7B0E090
:10017000BA93AA9325D12296D0C0AFE9B0E00C91F2
:1001800001FB00270EF401E041E0041709F0C5C0AF
:10019000009163000F3F09F004C080E08093A50048
:1001A00005C0A5EAB0E08C918F5F8C930091A5000B
:1001B000013009F0A5C0A3E6B0E08C919927909397
:1001C0004B0080934A00809163008093600000910F
:1001D0006000003081E008F480E08F9300916000BF
:1001E000053081E010F009F080E09F918923882399
:1001F00009F403C080E085BB83C000916000063035
:1002000081E008F480E08F9300916000083281E083
:1002100010F009F080E09F918923882309F403C03E
:1002200081E085BB6DC000916000093281E008F477
:1002300080E08F9300916000003581E010F009F0BC
:1002400080E09F918923882309F403C083E085BB64
:1002500057C000916000013581E008F480E08F9381
:1002600000916000083781E010F009F080E09F9174
:100270008923882309F403C087E085BB41C000912E
:100280006000093781E008F480E08F9300916000FE
:10029000003A81E010F009F080E09F9189238823E3
:1002A00009F403C08FE085BB2BC000916000013AC8
:1002B00081E008F480E08F9300916000083C81E0C9
:1002C00010F009F080E09F918923882309F403C08E
:1002D0008FE185BB15C000916000093C81E008F406
:1002E00080E08F93009160000E3F81E010F009F0F4
:1002F00080E09F918923882309F402C08FE385BBA6
:100300000091A500023009F008C0A3E6B0E08C918E
:10031000992790934900809348006894AFE9B0E032
:100320008C9186F98C93E894AFE9B0E08C9187F9D1
:100330008C93E7CEF894FFCF121201100100000059
:1003400008AAAA22EF0100010200010029090229DE
:100350000001010280FA0904000002030000000904
:1003600021110100012214000705810308000A077A
:1003700005020308000A140600FF0901A102090191
:10038000150025FF750895019102C00004040309BA
:1003900004000A0A0372006100640061006E00003C
:1003A0001C1C0352006100640061006E0020004CC0
:1003B00000450044002000760031002E003000008F
:1003C00080E08093A10080E6A881B9818C930091A0
:1003D0006300003809F03EC000916400063009F067
:1003E00038C000916600013009F007C0E8E3F3E08F
:1003F000F8D181E08093A1002CC0023009F007C041
:10040000ECE4F3E0EED181E08093A10022C0033060
:1004100009F01FC000916500003009F007C0ECE84A
:10042000F3E0DFD181E08093A10013C0013009F037
:1004300007C0E2E9F3E0D5D181E08093A10009C0D3
:10044000023009F006C0E0EAF3E0CBD181E080930E
:10045000A1006CC0003009F03AC000916400053082
:1004600009F021C0A881B981BA93AA935A924A92FD
:1004700080E0A42DB52D8C9381E0C5D113D12496B5
:1004800081E0BDD1A881B9810C9105FB00270EF454
:1004900001E040E0041709F001C0F4CF809165004D
:1004A0008093610013C0093009F010C0A881B981A0
:1004B000BA93AA935A924A9280E0A42DB52D8C93B8
:1004C00081E0A1D1EFD0249681E099D12FC00138ED
:1004D00009F011C000916400063009F00BC00091D2
:1004E0006600023209F006C0E6E7F3E07AD181E067
:1004F0008093A1001BC0013209F018C00091640074
:100500000A3009F013C081E08093A400A881B9816A
:10051000BA93AA935A924A9280E0A42DB52D8C9357
:1005200081E071D1BFD0249681E069D10091A10012
:10053000013009F00AC0A881B981BA93AA93A9E64B
:10054000B0E0BA93AA9302D02496089581E07ED1B8
:1005500081E07CD181E07AD182E078D145D1AE8151
:10056000BF81EBD20C923DD1AE81BF814C91A88569
:10057000B9850C91041708F006C0A885B9858C913F
:10058000AE81BF818C9382E0AC81BD818C9381E090
:10059000AA81BB818C93AE81BF814C91AA81BB8122
:1005A0000C91041710F009F077C0AC81BD818C91DB
:1005B0008F5F8C9319D1AC81BD81AD90BB24AA858E
:1005C000BB85AA0DBB1D1197B8D20C920AD1AC8184
:1005D000BD810C910A3081E009F080E08F93AE81FB
:1005E000BF814C91AA81BB810C91041781E009F075
:1005F00080E09F91892B882309F447C0AC81BD819D
:100600008C9182508C93AA85BB85BA93AA935A92F7
:100610004A92A885B9858C91A42DB52D8C9381E043
:10062000F2D040D0249681E0EAD0AA85BB850C9117
:1006300005FB00270EF401E040E0041709F021C09B
:1006400080E090E0A881B9818D939C93A0E3B0E015
:100650000C9103FB00270EF401E040E0041709F0C1
:100660000FC0A881B981D3D0A881B9810D911C9107
:10067000083E53E0150709F002C097D00DC0E6CF41
:10068000D4CF82E0AC81BD818C93AA81BB818C9157
:100690008F5F8C9308F47FCF85E0481A8827580A2B
:1006A00028960895AA81BB818C91807C8C9380E0F0
:1006B00090E0ADE9B0E08D939C93A881B9810C9155
:1006C000003009F41BC081E08A9381E08A93AA81FB
:1006D000BB818C918A934FEF5FEF25E030E8AD80CE
:1006E000BE80A2E0B0E0AA0DBB1D2BD2ADE9B0E008
:1006F0004D935C93ADE9B0E042E079D0A881B98137
:100700008C918D5F8C93AA81BB810C91A881B9815A
:100710004C91040FAA81BB810C93ADE9B0E08C91A0
:10072000A881B981AD90BB24AA81BB81AA0DBB1D54
:1007300011978C93A881B9818C918F5F8C93ADE9CF
:10074000B0E011968C91A881B981AD90BB24AA81AB
:10075000BB81AA0DBB1D11978C938BE4AA80BB8033
:10076000A1E0B0E0AA0DBB1D8C93AA81BB810C91C6
:1007700006FB00270EF401E040E0041709F008C072
:1007800083ECAA80BB80A1E0B0E0AA0DBB1D8C93D6
:100790006894AA81BB818C9184F98C93E894AA8196
:1007A000BB818C9185F98C9308956894AFE9B0E092
:1007B0008C9186F98C93E894AFE9B0E08C9187F93D
:1007C0008C9380E28093790080E28093850080E2C0
:1007D0008093910080E08093610080E08093A4008A
:1007E00008958E2E9F2E0895E82DF92D0895EA2F55
:1007F000FB2F8D91809581934A95D9F70895481ADA
:100800008827580A0895480E8827581E0895ED91A4
:10081000FC91EF5FFF4FFC93EE9308953197F1F752
:100820000895689462F80895E89462F80895EF9343
:10083000FF93EE27E82BE92B31F0E8EBFBE0319753
:10084000F1F70197D1F7FF91EF9108955A924A92EB
:10085000480E8827581E0895AF93BF934F930F9368
:100860001F932F933F933FB73F933395839BE9F7B4
:10087000829907C0839B05C0829903C0839B01C0F6
:100880007EC0A2E6B0E030919F00442736FF4BE0E7
:10089000A40F40E0B41F8399EBCF2FE704E03FEFB4
:1008A00000C0000010B300C004C010B332273D9355
:1008B0003FEF012702FB20F900B3297FA1F10C7063
:1008C00089F1102712FB21F910B30000237F89F171
:1008D0000000012702FB22F900B3277E81F11027D7
:1008E00012FB23F92F7C89F110B3012702FB24F9B5
:1008F00000C02F7979F100B32F774395102712FBB1
:1009000025F92F7361F110B3012702FB26F922307C
:1009100058F14C30A0F500B3102712FB27F9243012
:1009200040F1C3CF39C021603E7F1095000000B375
:10093000C6CF22603D7F009510B30000C9CF2B7F4A
:1009400034601095000000B3CACF2860377F00954F
:1009500000C0CACF20613F7E109500C0CCCF20627E
:100960003F7D009500C0CFCF20643F7B109500C035
:10097000D2CF20683F77009500C000C096CF3AB72D
:1009800036FD73CF3F913FBF3F912F911F910F9144
:100990004F91BF91AF91189530E43ABFA41BB0407E
:1009A0000D91102F13731132C1F41D912D914091AF
:1009B0006100110F221F16952F70141771F509365B
:1009C00049F0013E61F130919F0036FF26C00D32A3
:1009D00029F123C02093A00049F02091A00025FD1B
:1009E000CECF30919F00307C322B2F70A9E7B0E042
:1009F000203049F0A5E8B0E0213029F0A1E9B0E0CD
:100A0000223009F00AC01D91093691F0033CB9F07B
:100A10000B34A9F0023D31F0B2CF20622061209367
:100A2000A000ADCF1F7E106230E413271E93A7CF26
:100A300014FF03C0412F4F7022C01AE50BC0433092
:100A400041F036FFFACF30683F7B30939F004093F0
:100A5000780012EDBB27A1E141E011C052BB279500
:100A600020F43A9521F4220FF9CF502736E000C048
:100A700052BB2795B8F43A95B9F4220FF9CF5F939A
:100A80004F930CE0939A21B32C6021BB52B320E426
:100A9000502736E0000052BB279578F43A9579F458
:100AA000220FF9CF502736E02D9152BB27958EF1BA
:100AB00078F73A9579F7220FF9CF502736E000C042
:100AC00052BB279520F43A9521F4220FF9CF5027F5
:100AD00036E000C052BB279520F43A9521F4220F4E
:100AE000F9CF502736E000C052BB279520F43A9545
:100AF00021F4220FF9CF502736E04A9547FB52BB2D
:100B0000279520F43A9521F4220FF9CF502736E0AB
:100B1000A5CF00C022B3237F22BB4F91A41BB040BE
:100B2000422F286031B3337F00E40ABF5F910E91FA
:100B3000037422BB31BB42BB22CFC8953196002043
:100B4000089579910D919981903009F013D0502733
:100B500088E0440F551F10F4422753278A95C9F7A0
:100B60007A9581F789919991803019F08A0105D0A1
:100B7000A801089588E0112701C080E1F801F695E9
:0C0B8000E795001F111F8A95D1F708951A
:00000001FF
